:020000040000FA
:2B000000FFFF62FF2500FFFFFFFFFFFFFFFFFFFFFFFFFFFFFFFFFFFFFFFFFFFFFFFFFFFFFFFFFFFFFFFFFFFFFFFFFF76
:2B002B006018866118DCC11DDC61198665588665198601000000001886C11DDCC11D067770876118866118866100C488
:2B00560040100441100AA1100AE11084433884E3100401000000001004A1100AA1108442280441100441100441808349
:2B008100000000000000000000000000000000000000000000000000000000000000000000000000000000000080E7ED
:2B00AC00000000000000000000000000000000000000000000000000000000000000000000000000000000000080E7C2
:2B00D700000000000000000000800000022410820000000000000000000000000000000000000000000000000080B096
:2B010200000000000000000000001080040800800000000000000000000000000000000000000000000000000000EACC
:2B012D00080000000000000000000000000000000000000000000000000000000000000000000000000000000080EF30
:2B015800000000000000000000000000000000000000000000000000000000000000000000000000000000000080E715
:2B018300000000000000000000000000000000000020000000000000000000000000010000000000000000000080C4EC
:2B01AE00000000000000000000000000000000000000000000000000000000000000010000000000000000000080E6BF
:2B01D900000000000000000000000000000000000040000000000000000000000000000000000000000000000080A398
:2B020400000000000000000000000000000000000008000000000000000000000000000000000000000000000000EFD8
:2B022F00000000000000000000000000000000000000000000000000000000000000000000000000000000000080E73D
:2B025A00000000000000000000000000000000000040000000000000000000000000000000000000000000000080A316
:2B028500000000000000000000000000000000000000100000000000000000000000000000000000000000000080F7C7
:2B02B000000000000000000000000000000000000000000000000000000000000000400000000000000000000080A7BC
:2B02DB00000000000000000000000000000000000000010000000000000000000000000000000000000000000080E691
:2B030600000000000000000000000000000000000000000000000000000000000000000000000000000000000080E765
:2B033100000000000000000000000000000000000008000000000000000000000000000000000000000000000000EFAA
:2B035C00000000000000000000000000000100000000000000000000000000000000000000000000000000000080F6FF
:2B038700000000000002200004000000000080000000000000000000004000022000C01010000000000000000080FBE8
:2B03B200020000000002200004000000000008000000000000000000000000000000800010000000000000000008BC9C
:2B03DD00000000000000000000000000000000000000000000000000000000000000000000000000000000000080E78E
:2B040800000000000000000000000000000000000000000000000000004000022000000000000000000000000080E304
:2B043300000000000000000000000000000088020000000000000000000000000000401400000000000000000080E858
:2B045E00000000000000000000000000000000000000000000000000000000000000000000000000000000000080E70C
:2B048900020000000000000000000000000000000000000000000000000000000000000000000000000000000008ED51
:2B04B400800008800008800008800008800008800008000000000020000220000220000220000220000220000280E7BA
:2B04DF00800008800008800008800008800008800008000000000020000220000220000220000220000220000280E78F
:2B050A000000000000000000000000000000000000000000000000000000000000A0000000000000000000000000C561
:2B053500020000000000000000000000E0090000003E080000000000000000000018000000000000000000000080D6FC
:2B056000020000000000000000000000004100000000000000000000000000000040000000000000000000000008BC29
:2B058B00040000000000000000000000C00100000004010000000000000000000090040000000000000000000008E6F9
:2B05B600020000000000000000000000000000000000040000000000000000000000000000000000000000000008E923
:2B05E100020000000000000000000000000A000000200000000000000000000000A0080000000000000000000008C74C
:2B060C00020000000000000000000000000101000000000000000000000000000000400000000000000000000080A45B
:2B06370000000000000000000000000000030000001800000000000000000000004000000000000000000000000089B4
:2B066200000000000000000000000000001000000008000000000000000000000000000000000000000000000000EE67
:2B068D00000000000000000000000000600200000026020000000000000000000000000000000000000000000080E553
:2B06B800020000000000000000000000004000000010010000000000000000000000000000000000000000000008F9C3
:2B06E300000000000000000000000000400200000024000000000000000000000000000000000000000000000080E71F
:2B070E00000000000000000000000000800100000000080000000000000000000000000000000000000000000000F641
:2B073900000000000000000000000000800100000028000000000000000000000000000000000000000000000080D498
:2B076400000000000000000000000000000000000000100000000000000000000000000000000000000000000080F7E3
:2B078F00020000000000000000000000000000000010000000000000000000000000000000000000000000000008FC29
:2B07BA00000000000000000000000000001000000020000000000000000000000000000000000000000000000080C4A0
:2B07E500000000000000000000000000600000000006000000000000000000000000000000000000000000000080E71C
:2B081000000000000000000000000000000000000018040000000000000000000000000000000000000000000000FAA7
:2B083B00000000000000000000000000400001000024000000000000000000000000000000000000000000000080D5D8
:2B086600020000000000000000000000000000000000000000000000000000000000000000000000000000000008ED70
:2B089100020000000000000000000000002000000000010000000000000000000000000000000000000000000008EE23
:2B08BC00020000000000000000000000000000000000000000000000000000000000000000000000000000000008ED1A
:2B08E700020000000000000000000000000500000018000000000000000000000000000000000000000000000088A19E
:2B091200000000000000000000000000000100000008000000000000000000000020000000000000000000000000DCB5
:2B093D00000000000000000000000000E02200000006020000000000000000000098200000000000000000000000F4D9
:2B096800000000000000000000000000800100000010000000000000000000000040080000000000000000000000A3E8
:2B099300000000000000000000000000C01300000024010000000000000000000090000000000000000000000080EF42
:2B09BE00020000000000000000000000800100000000080000000000000000000000000000000000000000000088FCFF
:2B09E9000200000000000000000000008083000000280000000000000000000000A0080000000000000000000000D638
:2B0A1400040000000000000000000000800100000000100000000000000000000000400000000000000000000000AA38
:2B0A3F00020000000000000000000000808100000010000000000000000000000040000000000000000000000000A198
:2B0A6A00020000000000000000000000000100000000000000000000000000000000000000000000000000000080F4EA
:2B0A9500020000000000000000000000E04200000006040000000000000000000000000000000000000000000088C7B9
:2B0AC000000000000000000000000000802100000080000000000000000000000000000000000000000000000080FC6E
:2B0AEB00000000000000000000000000C00300000024000000000000000000000000000000000000000000000000FEFB
:2B0B1600000000000000000000000000800100000000000000000000000000000000000000000000000000000000FE35
:2B0B41000200000000000000000000008081000000A0000000000000000000000000000000000000000000000080D690
:2B0B6C00020000000000000000000000800300000000000000000000000000000000000000000000000000000088D67B
:2B0B9700040000000000000000000000800100000018000000000000000000000000000000000000000000000008EBA3
:2B0BC200020000000000000000000000000000000000020000000000000000000000000000000000000000000008EF0D
:2B0BED00020000000000000000000000600600000026000000000000000000000000000000000000000000000008A99E
:2B0C1800020000000000000000000000001000000080000000000000000000000000000000000000000000000000E43B
:2B0C4300000000000000000000000000400200000004000000000000000000000000000000000000000000000080C5FB
:2B0C6E00000000000000000000000000804100000000000000000000000000000000000000000000000000000000FAA0
:2B0C9900000000000000000000000000000200000080000000000000000000000000000000000000000000000000C5E9
:2B0CC400020000000000000000000000800100000000000000000000000000000000000000000000000000000088F406
:2B0CEF00000000000000000000000000800100000018000000000000000000000000000000000000000000000080E7DA
:2B0D1A00000000000000000000000000000400000010000000000000000000000040000000000000000000000080F6E4
:2B0D4500000000000000000000000000E0010000000E0200000000000000000000B84000000000000000000000808F8B
:2B0D70000000000000000000000000000081000000180000000000000000000000E000000000000000000000008081DE
:2B0D9B00020000000000000000000000C0030000001C100000000000000000000070000000000000000000000008A81C
:2B0DC60000000000000000000000000000000000001800000000000000000000006000000000000000000000000098F2
:2B0DF100000000000000000000000000000A000000381000000000000000000000E00400000000000000000000008C15
:2B0E1C00000000000000000000000000000101000010000000000000000000000040400000000000000000000080F3A6
:2B0E47000000000000000000000000000003000000280100000000000000000000A0000000000000000000000080DD57
:2B0E7200020000000000000000000000800500000010000000000000000000000040000000000000000000000088E511
:2B0E9D00020000000000000000000000E0000000000E1000000000000000000000B8200000000000000000000008E664
:2B0EC8000200000000000000000000008001000000180000000000000000000000600000000000000000000000088B71
:2B0EF300020000000000000000000000C0080000003C0200000000000000000000F0400000000000000000000008EBA9
:2B0F1E00000000000000000000000000801100000018010000000000000000000060400000000000000000000080C11D
:2B0F49000000000000000000000000008002000000380000000000000000000000E00000000000000000000000009053
:2B0F7400000000000000000000000000804100000010000000000000000000000040080000000000000000000000A792
:2B0F9F000200000000000000000000008003000000281000000000000000000000A00000000000000000000000A8EC36
:2B0FCA00020000000000000000000000000000000000000000000000000000000000000000000000000000000028CF03
:2B0FF500000000000000000000000000000000000000000000000000000000000000000000000000000000000080E76A
:2B102000800008800008800008800008800008800008000000000020000220000220000220000220000220000280E742
:2B104B00800008800008800008800008800008800008000000000020000220000220000220000220000220000280E717
:2B107600000000000000000000000000000000020022090000000000000000000010010000000000000000000080FE93
:2B10A100000000000000000000000000000000000000000000000000000000000000000000000000000000000080E7BD
:2B10CC00200002200000000000000000000000000000000000000008000000000000000000000010000000800080D6C9
:2B10F700000800000000000000000020000000000000000000000000000000000000000000000000002000022000C79D
:2B112200200802200000000000000020802000020022090000000008000000000010010000000010002000822080E51B
:2B114D00000000000000000000000000800001000000000000000000000000000020000000000000000000000000DDF9
:2B117800000000000000000000000000800000000000100000000000000000000000000000000000000000000000FFBD
:2B11A300000000000000000000000000002800000000080000000000000000000000000000000000000000000000ED04
:2B11CE00000000000000000000000000008000000000000000000000000000000000000000000000000000000080EF07
:2B11F900180000000000000000000000404000000004040000000000000000000000100000000000000000000080EFAC
:2B122400000000000000000000000000000000000080040000000000000000000000000000000000000000000000E338
:2B124F00000000000000000000000000000000000000000000000000000000000000000000000000000000000080E70D
:2B127A00080000000000000000000000000000000000000000000000000000000000000000000000000000000080EFD2
:2B12A500000000000000000000000000000000000010000000000000000000000000000000000000000000000080F698
:2B12D000100000000000000000000000004000000000000000000000000000000000000000000000000000000080F330
:2B12FB00000000000000000000000000000200000000000000000000000000000010200000000000000000000080F422
:2B1326000000000000000000000000000014000000000000000000000000000000002000000000000000000000808266
:2B135100000000000000000000000000000400000000000000000000000000000000000000000000000000000080A34A
:2B137C00000000000000000000000000000800000000000000000000000000000000000000000000000000000000E757
:2B13A700000000000000000000000000000000000000000000000000000000000000000000000000000000000080E7B4
:2B13D200000000000000000000000400000000000000000000000000000000000000000000000000000000000080A3C9
:2B13FD00000000000000000000000000000000000000000000000000000000000000000000000000000000000080E75E
:2B142800000000000000000000000000000000000000000000000000000000000000000000000000000000000080E732
:2B145300000000000000000000000000000000000000000000000000000000000000000000000000000000000080E707
:2B147E00020000000000000000000000000000000000000000000000000000000000000000000000000000000080E5DC
:2B14A900000000000000000000000000000000000000000000000000000000000000000000000000000000000080E7B1
:2B14D400000000000000000000000000000000000000000000000000000000000000000000000000000000000080E786
:2B14FF00000000000000000000000000000000000000000000000000000000000000000000000000000000000080E75B
:2B152A00000000000000000000000000000000000000000000000000000000000000000000000000000000000080E72F
:2B155500000000000000000000000000000000000000000000000000000000000000000000000000000000000080E704
:2B158000000000000000080000000000000000000000000000000000000000000000000000000000000000000080EFC9
:2B15AB00000000000000000000000020000000000200000000000000000000000000000000000000000000000080E78C
:2B15D600000000000000000000000210000200000100000000000000000000000000000000000000000000000080E76E
:2B160100000000000000000000000404000100000000000000000000000000000000000000000000000000000080F243
:2B162C00020000800000000000002000000000000000020000000000000000000000000000000000000000000000ED02
:2B165700000000000000000000000000000000004000000000000000000000000000000000000000000000000008EB35
:2B168200000000000000000000000000000100000000000000000000000000000000000000000000000000000008FE36
:2B16AD00000000800000000000002504000000000000020000000000000000000000000000000000000000000088F2ED
:2B16D800000000000000000000000000000000000000000000000000000000000000000000000000000000000008EFF0
:2B170300020000000000000000000000000000000000000000000000000000000000000000000000000000000080E554
:2B172E00800008800008800008800008800008800008000000000020000220000220000220000220000220000280E72D
:2B175900800008800008800008800008800008800008000000000020000220000220000220000220000220000280E702
:2B178400000000000000000000000000040000000100000000000000000000000000000000000000000000000080F2C3
:2B17AF000000000000000000000000066008006009000000000000000000000000000000000000000000000000089E92
:2B17DA00020000000000000000000000800100800100000000000000000000000000000000000000000000000080E57B
:2B18050002000000000000000000001C420A00C00B00000000000000000000000000000000000000000000000080A75C
:2B183000020000000000000000000000822100800100000000000000000000000000000000000000000000000080E502
:2B185B00020000000000000000000000000000000101000000000000000000000000000000000000000000000080E4FA
:2B188600000000000000000000000018800100800500000000000000000000000000000000000000000000000088B2DF
:2B18B100000000000000000000000000000000800300000000000000000000000000000000000000000000000000DCAD
:2B18DC00000000000000000000000010010000000000000000000000000000000000000000000000000000000080F759
:2B1907000000000000000000000000166000016008000000000000000000000000000000000000000000000000008650
:2B193200020000000000000000000010040000000000000000000000000000000000000000000000000000000080F004
:2B195D0000000000000000000000001C408000400001000000000000000000000000000000000000000000000088AE0C
:2B1988000000000000000000000000508003000000000000000000000000000000000000000000000000000000888158
:2B19B300000000000000000000000030000000000000000000000000000000000000000000000000000000000008DCF5
:2B19DE00000000000000000000000010000000800100000000000000000000000000000000000000000000000088E7DE
:2B1A0900020000000000000000000090000000800100000000000000000000000000000000000000000000000080ED32
:2B1A3400000000000000000000000018010000000000000000000000000000000000000000000000000000000000FF6F
:2B1A5F00000000000000000000000006E00900600B00000000000000000000000000000000000000000000000000AD55
:2B1A8A00000000000000000000000000840500801100000000000000000000000000000000000000000000000080A6F1
:2B1AB500020000000000000000000004C00300C00300000000000000000000000000000000000000000000000008ADC5
:2B1AE000020000000000000000000000800101800100000000000000000000000000000000000000000000000080F561
:2B1B0B00040000000000000000000000820300808300000000000000000000000000000000000000000000000080E9BA
:2B1B3600020000000000000000000000800100800101000000000000000000000000000000000000000000000080F50A
:2B1B6100020000000000000000000000800100800300000000000000000000000000000000000000000000000080C70C
:2B1B8C00020000000000010000000000010000000000000000000000000000000000000000000000000000000008ED35
:2B1BB70000000000000600000000001E600001600201000000000000000000000000000000000000000000000000DC3F
:2B1BE200000000000000080000000050000000000000000000000000000000000000000000000000000000000080BA46
:2B1C0D0000000000002C00000000001C408000402000000000000000000000000000000000000000000000000080DEE6
:2B1C3800020000000020000000000000000200000000000000000000000000000000000000000000000000000080E5F8
:2B1C6300000000000028000000000058800100000000000000000000000000000000000000000000000000000088814C
:2B1C8E00000000000000100000000080000000800100000000000000000000000000000000000000000000000008E62C
:2B1CB900000000000028000000000038000000800100000000000000000000000000000000000000000000000088E7B0
:2B1CE400000000000000000000000018000000000100000000000000000000000000000000000000000000000088E74D
:2B1D0F00020000000000000000000006700001600301000000000000000000000000000000000000000000000080A6A6
:2B1D3A00000000000000000000000020000200000100000000000000000000000000000000000000000000000080F6E5
:2B1D6500000000000000000000000004400000400101000000000000000000000000000000000000000000000080A6A7
:2B1D9000000000000000000000000000040000800100000000000000000000000000000000000000000000000000FAA9
:2B1DBB00020000000000000000000020008100002100000000000000000000000000000000000000000000000008C56C
:2B1DE600020000000000000000000000002000000100000000000000000000000000000000000000000000000080F639
:2B1E1100040000000000000000000000000000000500000000000000000000000000000000000000000000000080B667
:2B1E3C00020000000000000000002000000200001000000000000000000000000000000000000000000000000080C403
:2B1E6700020000000000000000600206F00300600000000000000000000000000000000000000000000000000000ECA7
:2B1E9200020000000000000000008000840900000000000000000000000000000000000000000000000000000008F816
:2B1EBD00000000000000000000400024C00300C00101000000000000000000000000000000000000000000000080F79A
:2B1EE800000000000000000000000030800100008000000000000000000000000000000000000000000000000000C5D9
:2B1F1300000000000000000000000000808300000200000000000000000000000000000000000000000000000000F6A8
:2B1F3E00020000000000000000800180800100000000000000000000000000000000000000000000000000000088ED7F
:2B1F6900000000000000000000800100800100000000000000000000000000000000000000000000000000000008EF54
:2B1F9400000000000000000000002000000000001100000000000000000000000000000000000000000000000090E47D
:2B1FBF00000000000000000000600206700A00600100000000000000000000000000000000000000000000000088EE3E
:2B1FEA00000000000000000000008000840500000100000000000000000000000000000000000000000000000088AF8B
:2B201500020000000000000000400024C00100400101000000000000000000000000000000000000000000000088D7D8
:2B204000000000000000000000008020800100008100000000000000000000000000000000000000000000000000CD06
:2B206B00000000000000000000000200800100000300000000000000000000000000000000000000000000000000EFD5
:2B209600000000000000000000800108800100000500000000000000000000000000000000000000000000000000BA56
:2B20C100020000000000000000000000820100800100000000000000000000000000000000000000000000000080E787
:2B20EC00020000000000000000000000010000000100000000000000000000000000000000000000000000000008FDC0
:2B211700040000000000000000600406E00900600900000000000000000000000000000000000000000000000088A7AE
:2B214200020000000000000000008000000100800100000000000000000000000000000000000000000000000088EDF9
:2B216D00020000000000000000400204D00B00C00B00000000000000000000000000000000000000000000000008DF72
:2B219800020000000000000000000208040500800100000000000000000000000000000000000000000000000080877F
:2B21C300000000000000000000000020800100000101000000000000000000000000000000000000000000000000DD71
:2B21EE000000000000000000000020200021008005000000000000000000000000000000000000000000000000008957
:2B221900080000000000000000800000800100800100000000000000000000000000000000000000000000000050B20E
:2B224400000000000000000000000000000000000000000000000000000000000000000000000000000000000048AB7C
:2B226F00000000000000000000000000000000000000000000000000000000000000000000000000000000000080E7DD
:2B229A00800008800008800008800008800008800008000000000020000220000220000220000220000220000280E7B6
:2B22C500800008800008800008800008800008800008000000000020000220000220000220000220000220000280E78B
:2B22F000000000000000000000200222281400200080020000000000000000000000000000000000000000000000A8F9
:2B231B00000000000000000000000010004000000000000000000000000000000000000000000000000000000080F2D5
:2B234600000000000000000000000000000000000000000000000000000000000000000000000000000000000080E705
:2B237100000000000000000000000000000800800000000000000000000000000000000000000000000000000080EF4A
:2B239C000000000000000000002002322A5C00200080000000000000000000000000000000000000000000000080BD5F
:2B23C700000000000000000000400000402000000001000000000000000000000000000000000000000000000080F5D5
:2B23F2000000000000000000000000204100000080000000000000000000000000000000000000000000000000808CD3
:2B241D00000000000000000000000000000000000000000000000000000000000000000000000000000000000080E72D
:2B244800000000000000000000004080000000800000000000000000000000000000000000000000000000000080EBBE
:2B24730008000000000000000000000000400100C000000000000000000000000000000000000000000000000090E6BF
:2B249E00000000000004040000000000000000000000000000000000000000000000000000000000000000000090B2C9
:2B24C900000000000000000000000000000000000000000000000000000000000000000000000000000000000080E781
:2B24F400000000000010000000000000000000000000000000000000000000000000000000000000000000000080F637
:2B251F00000000000000000000000004100000000000000000000000000000000000000000000000000000000080B746
:2B254A00080000000000000000000000000000000000000000000000000000000000000000000000000000000080EFEF
:2B257500000000000000000000000000000000000000000000000000000000000000000000000000000000000080E7D4
:2B25A000020000000000000000002000008000004000000000000000000000000000000000000000000000000080EBC3
:2B25CB00000000000000000000000000000000000000000000000000000000000000000000000000000000000080E77E
:2B25F600000000000000000000000000000000000000000000000000000000000000000000000000000000000080E753
:2B262100000000000000000000000000000000000000000000000000000000000000000000000000000000000080E727
:2B264C00000000000000000000000000000000000000000000000000000000000000000000000000000000000080E7FC
:2B267700000000000000000000000000000000000000000000000000000000000000000000000000000000000080E7D1
:2B26A200000000000000000000000000000000000000000000000000000000000000000000000000000000000080E7A6
:2B26CD00120000000000000000000000000000000000000000000000000000000000000000000000000000000080F55B
:2B26F800000000000000000000000000000000000000000000000000000000000000000000000000000000000080E750
:2B272300000000000000000000000000000000000000000000000000000000000000000000000000000000000080E724
:2B274E00000000000000000000000000000000000000000000000000000000000000000000000000000000000080E7F9
:2B277900000000000000000000000000000000000000000000000000000000000000000000000000000000000080E7CE
:2B27A400120000000000000000000000000000000000000000000000000000000000000000000000000000000080F583
:2B27CF00000000000000000000000000000000000000000000000000000000000000000000000000000000000080E778
:2B27FA00000000000000000000000000000000000000000000000000000000000000000000000000000000000080E74D
:2B282500000000000000000000000000000000000000000000000000000000000000000000000000000000000080E721
:2B285000000000000000000000000000000000000000000000000000000000000000000000000000000000000080E7F6
:2B287B00000000200000000000000000000000008000000000000000000000000000000000000000000000000080CF43
:2B28A600020000000000000000000000000000000000000000000000000000000000000000000000000000000008ED10
:2B28D100020000000000000000000000000000000000000000000000000000000000000000000000000000000080E575
:2B28FC00040000200000000000000000000000008000000000000000000000000000000000000000000000000080CBC2
:2B292700020000000000000000000000000000000000000000000000000000000000000000000000000000000080E51E
:2B295200020000000000000000000000000000000000000000000000000000000000000000000000000000000080E5F3
:2B297D00020000000000000000000000000000000000000000000000000000000000000000000000000000000008ED38
:2B29A800800008800008800008800008800008800008000000000020000220000220000220000220000220000280E7A1
:2B29D300800008800008800008800008800008800008000000000020000220000220000220000220000220000280E776
:2B29FE00000000000000000000000000000000000000000000000000000000000000000000000000000000000080E747
:2B2A2900020000000000000000000000000000000000000000000000000000000000000000000000000000000008ED8B
:2B2A5400000000000000000000000000000000000000000000000000000000000000000000000000000000000080E7F0
:2B2A7F00000000000000000000000000000000000000000000000000000000000000000000000000000000000080E7C5
:2B2AAA00000000000000000000000000000000000000000000000000000000000000000000000000000000000080E79A
:2B2AD500000000000000000000000000000000000000000000000000000000000000000000000000000000000080E76F
:2B2B0000020000000000000000000000000000000000000000000000000000000000000000000000000000000008EDB3
:2B2B2B00000000000000000000000000000000000000000000000000000000000000000000000000000000000080E718
:2B2B5600000000000000000000000000000000000000000000000000000000000000000000000000000000000080E7ED
:2B2B8100000000000000000000000000000000000000000000000000000000000000000000000000000000000080E7C2
:2B2BAC00020000000000000000000000000000000000000000000000000000000000000000000000000000000008ED07
:2B2BD700000000000000000000000000000000000000000000000000000000000000000000000000000000000080E76C
:2B2C0200000000000000000000000000000000000000000000000000000000000000000000000000000000000080E740
:2B2C2D00000000000000000000000000000000000000000000000000000000000000000000000000000000000080E715
:2B2C5800000000000000000000000000000000000000000000000000000000000000000000000000000000000080E7EA
:2B2C8300020000000000000000000000000000000000000000000000000000000000000000000000000000000008ED2F
:2B2CAE00000000000000000000000000000000000000000000000000000000000000000000000000000000000080E794
:2B2CD900000000000000000000000000000000000000000000000000000000000000000000000000000000000080E769
:2B2D0400000000000000000000000000000000000000000000000000000000000000000000000000000000000080E73D
:2B2D2F00020000000000000000000000000000000000000000000000000000000000000000000000000000000008ED82
:2B2D5A00020000000000000000000000000000000000000000000000000000000000000000000000000000000080E5E7
:2B2D8500040000000000000000000000000000000000000000000000000000000000000000000000000000000080E3BC
:2B2DB000020000000000000000000000000000000000000000000000000000000000000000000000000000000080E591
:2B2DDB00020000000000000000000000000000000000000000000000000000000000000000000000000000000080E566
:2B2E0600020000000000000000000000000000000000000000000000000000000000000000000000000000000008EDAA
:2B2E3100000000000000000000000000000000000000000000000000000000000000000000000000000000000080E70F
:2B2E5C00000000000000000000000000000000000000000000000000000000000000000000000000000000000080E7E4
:2B2E8700000000000000000000000000000000000000000000000000000000000000000000000000000000000080E7B9
:2B2EB200020000000000000000000000000000000000000000000000000000000000000000000000000000000008EDFE
:2B2EDD00020000000000000000000000000000000000000000000000000000000000000000000000000000000080E563
:2B2F0800040000000000000000000000000000000000000000000000000000000000000000000000000000000080E337
:2B2F3300020000000000000000000000000000000000000000000000000000000000000000000000000000000080E50C
:2B2F5E00020000000000000000000000000000000000000000000000000000000000000000000000000000000080E5E1
:2B2F8900020000000000000000000000000000000000000000000000000000000000000000000000000000000008ED26
:2B2FB400000000000000000000000000000000000000000000000000000000000000000000000000000000000080E78B
:2B2FDF00000000000000000000000000000000000000000000000000000000000000000000000000000000000080E760
:2B300A00000000000000000000000000000000000000000000000000000000000000000000000000000000000080E734
:2B303500020000000000000000000000000000000000000000000000000000000000000000000000000000000008ED79
:2B306000000000000000000000000000000000000000000000000000000000000000000000000000000000000008EF4E
:2B308B00000000000000000000000000000000000000000000000000000000000000000000000000000000000090F694
:2B30B600000000000000000000000000000000000000000000000000000000000000000000000000000000000008EFF8
:2B30E100000000000000000000000000000000000000000000000000000000000000000000000000000000000008EFCD
:2B310C00020000000000000000000000000000000000000000000000000000000000000000000000000000000008EDA1
:2B313700000000000000000000000000000000000000000000000000000000000000000000000000000000000080E706
:2B316200000000000000000000000000000000000000000000000000000000000000000000000000000000000080E7DB
:2B318D00000000000000000000000000000000000000000000000000000000000000000000000000000000000080E7B0
:2B31B800020000000000000000000000000000000000000000000000000000000000000000000000000000000008EDF5
:2B31E300000000000000000000000000000000000000000000000000000000000000000000000000000000000080E75A
:2B320E00000000000000000000000000000000000000000000000000000000000000000000000000000000000080E72E
:2B323900000000000000000000000000000000000000000000000000000000000000000000000000000000000080E703
:2B326400000000000000000000000000000000000000000000000000000000000000000000000000000000000080E7D8
:2B328F00020000000000000000000000000000000000000000000000000000000000000000000000000000000008ED1D
:2B32BA00000000000000000000000000000000000000000000000000000000000000000000000000000000000080E782
:2B32E500000000000000000000000000000000000000000000000000000000000000000000000000000000000080E757
:2B331000000000000000000000000000000000000000000000000000000000000000000000000000000000000080E72B
:2B333B00020000000000000000000000000000000000000000000000000000000000000000000000000000000008ED70
:2B336600020000000000000000000000000000000000000000000000000000000000000000000000000000000080E5D5
:2B339100040000000000000000000000000000000000000000000000000000000000000000000000000000000080E3AA
:2B33BC00020000000000000000000000000000000000000000000000000000000000000000000000000000000080E57F
:2B33E700020000000000000000000000000000000000000000000000000000000000000000000000000000000080E554
:2B341200020000000000000000000000000000000000000000000000000000000000000000000000000000000008ED98
:2B343D00000000000000000000000000000000000000000000000000000000000000000000000000000000000080E7FD
:2B346800000000000000000000000000000000000000000000000000000000000000000000000000000000000080E7D2
:2B349300000000000000000000000000000000000000000000000000000000000000000000000000000000000080E7A7
:2B34BE00000000000000000000000000000000000000000000000000000000000000000000000000000000000080E77C
:2B34E900000000000000000000000000000000000000000000000000000000000000000000000000000000000080E751
:2B351400800008800008800008800008800008800008000000000020000220000220000220000220000220000280E729
:2B353F00800008800008800008800008800008800008000000000020000220000220000220000220000220000280E7FE
:2B356A00000000000000000000000000000000000000000000000000000000000000000000000000000000000080E7CF
:2B359500000000000000000000000000000000000000000000000000000000000000000000000000000000000080E7A4
:2B35C000000000000000000000000000000000000000000000000000000000000000000000000000000000000080E779
:2B35EB00000000000000000000000000208000010000000000000000000000000000000000000000000000000080CEC6
:2B361600000000000000000000000000208000010000000000000000000000000000000000000000000000000080CE9A
:2B364100000000000000000000000000000000000000000000000000000000000000000000000000000000000080E7F7
:2B366C00000000000000000000000000000000000000000000000000000000000000000000000000000000000080E7CC
:2B369700000000000000000000000000000000000000000000000000000000000000000000000000000000000080E7A1
:2B36C200000000000000000000000000000000000000000000000000000000000000000000000000000000000080E776
:2B36ED000000000000000000000000000000000000000000000000000000000000000000000000000000000000A0C54D
:2B371800100000000000000000000000000000000000000000000000000000000000000000000000000000000080F7FF
:2B374300000000000000000000000000000000000000000000000000000000000000000000000000000000000080E7F4
:2B376E00000000000000000000000000000000000000000000000000000000000000000000000000000000000080E7C9
:2B3799000000000000000000000000000000000000000000000000000000000000000000000000000000000000A0C5A0
:2B37C400000000000000000000000000000000000000000000000000000000000000000000000000000000000080E773
:2B37EF00000000000000000000000000000000000000000000000000000000000000000000000000000000000080E748
:2B381A00020000000000000000000000000000000000000000000000000000000000000000000000000000000080E51C
:2B384500000000000000000000000000000000000000000000000000000000000000000000000000000000000080E7F1
:2B387000000000000000000000000000000000000000000000000000000000000000000000000000000000000080E7C6
:2B389B00000000000000000000000000000000000000010000000000000000000000000000000000000000000080E69B
:2B38C600000000000000000000000000000000000000020000000000000000000000000000000000000000000080E570
:2B38F100000000000000000000000000000000000000000000000000000000000000000000000000000000000080E745
:2B391C00000000000000000000000000000000000000000000000000000000000000000000000000000000000080E719
:2B394700A0280AA1100441100441100441100441108403000000002804411004411004411004412804A1108AA280BB47
:2B397200C075DDC11D8661188661188661188661188605000000007087611886611886611886617087C11D5CD705BD94
:02399D00FFFF2A
:00000001FF
